:020000040800F2
:1000000048080020D50000088914000819130008CA
:1000100000000000000000000000000000000000E0
:10002000000000000000000000000000C7170008EA
:100030000000000000000000D1140008C9170008EB
:100040000501000805010008050100080501000878
:100050000501000805010008050100080501000868
:100060000501000805010008050100080501000858
:100070000501000805010008050100080501000848
:100080000501000800000000000000000501000854
:10009000000000008D1800089D18000805010008E8
:1000A00000000000D5140008050100080501000843
:1000B0000501000800000000050100080501000816
:1000C0000348854600F06CF800480047052000080A
:1000D000480800200C4880F308880C480168090E85
:1000E0000B4A914205D10B480B4901600B480C4962
:1000F00001600C4880470C480047FEE7FEE7FEE73A
:10010000FEE7FEE7FEE700004808002004000000CC
:100110001F00000018100240010000000000014014
:100120000000000031180008C100000830B50B467F
:10013000014600202022012409E00D46D5409D42C1
:1001400005D31D469540491B254695404019154647
:10015000521E002DF1DC30BD03460B439B0703D03C
:1001600009E008C9121F08C0042AFAD203E00B787C
:100170000370401C491C521EF9D27047D2B201E0F4
:100180000270401C491EFBD270470022F6E710B5F2
:1001900013460A4604461946FFF7F0FF204610BDF5
:1001A000064C0125064E05E0E36807CC2B430C3CCA
:1001B00098471034B442F7D3FFF786FF8C24000829
:1001C000AC24000870B50024014620314A78022A88
:1001D00003D004218163012416E0026813680E2510
:1001E000AB431360026813685B085B001360012275
:1001F000056C1346AB40C56B6B604A7000220A70F9
:10020000416B002900D08847204670BD31B500F011
:10021000B3F8009C0546601C00D0641C00F0ACF8EC
:10022000401BA042FAD338BDF8B5002389E0012471
:100230009C402A46A44622407ED04C68022C01D025
:10024000122C0CD1DC08A40027183C6A5D07ED0EC7
:100250000F26AE40B4430E69AE4026433E620568A9
:100260005E000324B4400F79A543BF07BF0FB7401A
:100270002F4307604D68012D05D0022D03D0112DAD
:1002800001D0122D0ED18568CF68A543B7402F430A
:10029000876047686546AF430D79ED06ED0F9D40D9
:1002A0003D434560C568A5438C68B4402C43C46099
:1002B0004C68E40044D5264CA56901263543A56168
:1002C000A4699D0834400094224CAD002F19BC68ED
:1002D0009D072E0F0F25B540AC430925ED06A8421A
:1002E00001D100250AE01C4DA84201D1012505E0FD
:1002F0001A4DA84201D1022500E00525B54025434D
:10030000BD60174C25684E689543F60300D515432C
:10031000256065684E689543B60300D51543656052
:10032000A5684E689543F60200D51543A560E568BB
:100330004E689543B60200E002E000D51543E56043
:100340005B1C0A681546DA4000D070E7F8BD000073
:10035000001002400000014000040048000800486E
:100360000004014042694A4042617047002A01D0BE
:1003700081617047816270470148006870470000E2
:100380001400002070B5040005D025466035687A59
:10039000002802D006E0012070BD0020287220460F
:1003A00000F032FF24206872206801684908490083
:1003B0000160204601F08CFB0128EDD0606A002826
:1003C00002D0204601F0EBFA206841680922D202EF
:1003D00091434160206881682222914381602068B6
:1003E000816808221143816020680168012211435D
:1003F0000160204601F038FB70BD00000248016832
:10040000491C0160704700001400002010B5064828
:100410000168102211430160002000F007F800F08D
:1004200017F8002010BD00000020024010B504465F
:1004300000F0E8F87D21C900FFF778FE00F0C4FC69
:1004400000222146501E00F02FF8002010BD0000B1
:1004500008B50F488169012211438161816911400A
:100460000091C26901040A43C261C06900220840C8
:1004700000901146501F00F017F800221146901E00
:1004800000F012F800221146501E00F00DF808BDD1
:1004900000100240C106C90E0120884001490860D1
:1004A0007047000000E100E010B500F0EFFF10BD64
:1004B000F8B505464E480E460068C007C00FB0426A
:1004C0000AD24B480168490849003143016000687D
:1004D000C007C00FB04270D12878464C800705D5C0
:1004E0006068F0218843A968084360602878C007E5
:1004F00053D06868012817D0022818D0032819D0D3
:1005000021688907002958DA616889088900014350
:100510006160FFF731FF69680746012913D002299E
:100520001DD0032927D034E021688903EAE7216838
:100530008901E7E7616BC903E4E7FFF71DFFC11B12
:100540002D48814223D860680007800F0128F4D12C
:1005500023E0FFF711FFC11B2748814217D86068CD
:100560000007800F0228F4D117E0FFF705FFC11B39
:10057000214881420BD860680007800F0328F4D11E
:100580000BE0FFF7F9FEC11B1B48814201D9032094
:10059000F8BD60680007800FF3D115480168C907EE
:1005A000C90FB1420BD901684908490031430160C4
:1005B0000068C007C00FB04201D00120F8BD287804
:1005C000400706D56068072109028843E9680843A7
:1005D000606000F02DF86168084A0906090F515C57
:1005E000C840074908600020FFF720FF0020F8BD41
:1005F000002002400010024088130000732400080D
:100600001800002001480068704700001800002012
:100610000448054900684968044A4905490F515C86
:10062000C8407047180000200010024083240008D2
:1006300030B516A30FCB89B06C460FC417A30FCBF0
:100640000FC41A494A680C20144604401848042C68
:1006500005D0184B082C04D00C2C00D1184609B03A
:1006600030BD9402240F6D462C5DC96A04AD0907A4
:10067000090FD203695C920F022A02D0032A00D12B
:100680001846FFF753FD6043E9E700000203040545
:10069000060708090A0B0C0D0E0F101001020304C7
:1006A00005060708090A0B0C0D0E0F10001002407A
:1006B00000127A00006CDC02FEB504460078F04EB1
:1006C000F04DC00748D068680007800F01281FD090
:1006D00068680007800F022804D16868C003800F93
:1006E000022815D06168012919D001208004002951
:1006F00001D0052917D02968B143296029688143B1
:100700002960606800281BD0FFF736FE074613E01B
:100710002868800320D56068002876D01CE028680F
:1007200030432860EDE7296801432960F7E7FFF7C8
:1007300023FEC01B642869D828688003F7D50BE026
:10074000FFF71AFE074604E0FFF716FEC01B6428F9
:10075000F1D828688003F7D4207880073ED56868F0
:100760000007800F14D068680007800F022804D1AA
:100770006868C003800F01280AD0E0680028286854
:100780001DD0012108432860FFF7F6FD07460BE066
:10079000286880070BD5E068012836D107E0FFF70D
:1007A000EBFDC01B0228C6D828688007F7D528684B
:1007B000F82188432169C900084328600EE04008F9
:1007C00040002860FFF7D8FD074604E0FFF7D4FD9E
:1007D000C01B0228AFD828688007F7D4207800070C
:1007E00024D5E0690028686A11D0012108436862B5
:1007F000FFF7C2FD074604E0FFF7BEFDC01B02285D
:1008000099D8686A8007F7D510E036E1D1E0400852
:1008100040006862FFF7B0FD074604E0FFF7ACFD5B
:10082000C01B022887D8686A8007F7D4207804277D
:100830004007002861DA00200190E869C00008D470
:10084000E969B8060143E961E969014001200091C5
:1008500001908D480168C90511D4016882151143C2
:100860000160FFF789FD009005E0FFF785FD009925
:10087000401A642897D884480068C005F5D5A06858
:1008800001280AD0002801D0052811D0286A400884
:1008900040002862286AB84302E0286A0121084320
:1008A0002862A068002812D0FFF766FD00900AE0D9
:1008B000286A38432862F0E7FFF75EFD0099411A85
:1008C0007248814275D8286A8007F5D50DE0FFF798
:1008D00053FD009006E0FFF74FFD0099411A6B4869
:1008E000814266D8286A8007F5D40198002804D090
:1008F000E969012000078143E9612078C00635D508
:10090000606901280CD0401D686B24D038436863AF
:10091000686B400840006863FFF72EFD074622E041
:10092000686B38436863686B012108436863FFF7AD
:1009300023FD074604E0FFF71FFDC01B022838D83F
:10094000686B8007F7D5686BF8218843A169C900F7
:10095000084368630AE0B8436863F4E7FFF70CFDF7
:10096000C01B022825D8686B8007F7D42078800642
:1009700037D568680007800F032813D06868000720
:10098000800F022804D16868C003800F032809D0B3
:10099000206A0028686B16D030436863FFF7ECFCD0
:1009A00006460CE0686BC0031BD5206A012864D1A1
:1009B00017E05BE0FFF7E0FC801B022856D8686B6D
:1009C000C003F7D50DE0B0436863FFF7D5FC0646DA
:1009D00004E0FFF7D1FC801B022847D8686BC003F6
:1009E000F7D4606A002846D069680907890F022990
:1009F00043D0012636060228286805D0B043286077
:100A0000FFF7BAFC044633E0B0432860FFF7B4FCBC
:100A1000074604E0FFF7B0FCC01B022826D8286870
:100A20008001F7D4E86A216B000900010843E862FD
:100A3000A16AE06A084369687B22D20391430843B4
:100A40006860286830432860FFF796FC044604E09D
:100A5000FFF792FC001B022808D828688001F7D510
:100A600009E0FFF789FC001B022801D90320FEBD25
:100A700028688001F5D40020FEBD0120FEBD0000E5
:100A800000000100001002400070004088130000C8
:100A900070470000F8B504460068426881684B065C
:100AA00005D4CB0703D0530601D5E16C04E08B07D6
:100AB00005D5130603D5216D20468847F8BDFF23D1
:100AC00061331942FAD09306F8D523464D064033D8
:100AD000002D09DA5D7F032D3CD0256E04263543B9
:100AE0002566C568856800958E060125002E08DA02
:100AF000266E2E4326668668009606684027BE430B
:100B00000660C80506D5206E0821084320662068C7
:100B100080680090206E0028D0D020684168E026D0
:100B2000B14341605D77900718D02068416889081B
:100B300089004160A06D0B4D002803D04563A06D76
:100B4000FFF740FB606D0028B8D04563606DFFF78C
:100B500039FBF8BDC16880680090F8BD2046FFF7FA
:100B600097FFF8BD47160008F8B5040007D0002627
:100B700025464035A662687F002802D005E00120A6
:100B8000F8BD2E77204600F04BF802236B772068E3
:100B900001684022914301600721E0680902884210
:100BA00001D9002201E0012212030F273F02B842BF
:100BB00002D0884200D0A662276B002F05D1884260
:100BC00001D9236301E001202063A16860686369A3
:100BD00008432169194308430123A1695B021940B5
:100BE0000843E1690843216A0843A16A0843216870
:100BF0000860616B606AA36908431B0C0427E16805
:100C00003B40194308432168104348602068C1698C
:100C10007A029143C1612666012068770020F8BD01
:100C200000B50068114987B088421DD1104882691B
:100C300081140A438261806908400590F020009089
:100C400002200190002103200390029104910920C9
:100C50006946C006FFF7E8FA002211461920FFF79F
:100C600023FC1920FFF716FC07B000BD003001403F
:100C70000010024070470000F0B504468C46403436
:100C8000217F0025C768964601290CD001212177D4
:100C9000667F4168012E0CD0CA1FFD3A07D18168DA
:100CA000002904D101E00220F0BD042E01D002256C
:100CB00040E0614600291BD07146002918D0002B66
:100CC00016D0617F042901D00521617700210166DA
:100CD000614681638387C38771460164A380E38093
:100CE000072109028F4205D9144AC264144A04E05C
:100CF00001251FE0134AC264134A02650122120350
:100D00008F4202D8E188022903D301684B689343DC
:100D100002E001684B6813434B6001684A68E023B6
:100D20001A434A6000680168490603D401684022FA
:100D300011430160002020772846F0BDE51400082B
:100D4000791500081B150008AD15000870B50122C3
:100D5000124E150229463046FFF708FB104C20784A
:100D6000DE2802D00F49012048700D4801F072FAC8
:100D7000A078032805D1092000220221C006FFF730
:100D8000F5FA074A2023D11A0748FFF775FF00221A
:100D900029463046FFF7EAFA70BD0000000400481B
:100DA000DC01002004000020280000200422044967
:100DB0000428086902D09043086170471043FBE79C
:100DC00000E000E070470000094910B5401E88426D
:100DD00001D9012010BD074C60610321081F00F0FC
:100DE00055FB0020A06107202061002010BD0000FD
:100DF000FFFFFF0000E000E010B5FFF7E3FF10BDCC
:100E00007047704770B502462032137F012B1BD00C
:100E10000123137702245477046865687026B5436C
:100E20006560046865680E68354365600468A56898
:100E30008026B543A5600068846849680C438460D7
:100E400053770020107770BD022070BD70B504008C
:100E500005D025462035687F002802D006E0012015
:100E600070BD00202877204600F00AF8022068773D
:100E7000211D206800F01AFD01206877002070BD58
:100E800008B50122016892071848914207D1C1694B
:100E900001221143C161C0691040009008BD144A8D
:100EA00091420ED18269012149040A43826180691D
:100EB00000220840009011461520FFF7F5FA152092
:100EC00010E00C4A9142E9D18269012189040A4368
:100ED0008261806900220840009003211620FFF7FC
:100EE000E3FA1620FFF7D6FA08BD00000010024012
:100EF00000440140004801400222014620314A7767
:100F0000026813680120034313604877002070478C
:100F10000268D36801210B43D360006802680A436A
:100F2000026000207047F8B5054604462035287F4A
:100F3000012817D001272F77022068772268906850
:100F40007726FF23B0431B0298439060086850281F
:100F500037D00EDC202857D006DC00284ED01028D1
:100F600040D14EE00220F8BD302850D0402839D181
:100F70003CE060282DD0702817D001221203801A7F
:100F80000ED090422ED1CB684A688968206800F064
:100F9000CFFC20688168012292031143816021E027
:100FA00020688168C908C900F8E7CB684A68896881
:100FB000206800F0BDFC21688868B0433043886039
:100FC00010E0CA684968206800F0C5FC502120681C
:100FD00006E0CA684968206800F0CEFC60212068FD
:100FE00000F0B1FC6F7700202877F8BDCA68496827
:100FF000206800F0B0FC40212068F1E70021206863
:10100000EEE710212068EBE720212068E8E7302197
:101010002068E5E7704770B504460068016900255F
:10102000C9438907002915DBC168C943890711D461
:10103000E91E016101202077206880698007204631
:1010400002D0FFF7E7FF04E000F096F8204600F03A
:1010500094F8257720680169C943490717D4C16806
:10106000C943490713D40421C943016102202077F1
:10107000206880698005800F204602D0FFF7CAFFF4
:1010800004E000F079F8204600F077F82577206832
:101090000169C943090716D4C168C943090712D4B5
:1010A0000821C9430161042020772068C0698007B6
:1010B000204602D0FFF7AEFF04E000F05DF82046C6
:1010C00000F05BF8257720680169C943C90617D489
:1010D000C168C943C90613D41021C943016108205E
:1010E00020772068C0698005800F204602D0FFF776
:1010F00091FF04E000F040F8204600F03EF825772C
:1011000020680169C943C90708D1C168C943C90733
:1011100004D1891E0161204600F030F82068016981
:10112000C943090609D4C168C943090605D4802109
:10113000C94301612046FFF763FE20680169C94386
:10114000490609D4C168C943490605D44021C943A9
:101150000161204600F056F820680169C9438906FC
:1011600009D4C168C943890605D42021C943016156
:101170002046FFF746FE70BD70477047F8B505463C
:101180001D4809270646FF06403E1C4C85421AD1E1
:10119000012149023846FFF7E5F82046083001F002
:1011A00036F8002820D00021415E084600F060FE9D
:1011B0002046083001F036F800F09CFE606000F038
:1011C0006DFE3168C862B5420DD1606800280AD052
:1011D000012189023846FFF7C5F8606800280848F1
:1011E00006DD01F0BAF8F8BD002000F041FEE3E7AB
:1011F00001F0AAF8F8BD00000C0100200400002056
:10120000340200207047000000B500680E4987B026
:10121000884216D10D48C269012149040A43C261BE
:10122000C06908400590042000901220019001211F
:10123000032003900291049109206946C006FEF73D
:10124000F3FF07B000BD0000004400400010024062
:10125000FFB5064604466036707A83B00D462028F6
:1012600058D1002D0CD00598002809D00120A16884
:101270000003814207D12069002804D1E80702D089
:10128000012007B0F0BD307A012843D00120307230
:101290000020E06621207072FFF76EF8019027466B
:1012A0004037059838820598788218E0788A401E81
:1012B000788206980090002280212046019B00F051
:1012C0009FFC002818D10120A1680003814202D1AF
:1012D0002069002812D02168287808856D1C788A3A
:1012E0000028E3D106980090002240212046019B6F
:1012F00000F086FC002808D00320C2E72888216877
:10130000C005C00D0885AD1CE9E7202070720020E3
:101310003072B6E70220B4E7FEE70000F0B52448DB
:1013200087B04269012189040A43426142690A4047
:101330000592426909010A43426142690A400592E5
:10134000426949110A43426140691A4F08404C12F0
:101350000590002221463846FFF708F800220321B5
:101360001548FFF703F8154E092000223146C00644
:10137000FEF7FCFF009400240125019502946946C4
:1013800038460394FEF750FF03200090029469460C
:10139000019503940848FEF747FF09200294694627
:1013A000C006009601950394FEF73EFF07B0F0BD1E
:1013B000001002400004004800140048020600002B
:1013C00010B50D480B490160002141608160016149
:1013D000416181610722016212024162C260816241
:1013E00007220163C2624163FFF7BEFB002800D001
:1013F000FEE710BD003001402800002010B501219B
:10140000124886B08907016000242F218460416062
:101410000461611E8461C160FFF718FD002800D0DF
:10142000FEE701200003009069460848FFF77BFDB6
:10143000002800D0FEE7049404A904480594FFF7AF
:10144000E1FC002800D0FEE706B010BD8C000020B3
:1014500010B50C480A490160E121490241600021B0
:101460008160C16001618161C161082201624261E4
:101470004162FEF787FF002800D0FEE710BD0000A4
:10148000004400404C010020704700008307FF2209
:10149000DB0E9A408907090E994000280BDA0007F5
:1014A000000F0838830808489B001818C369934345
:1014B0000B43C3617047830804489B001B181868DE
:1014C000904308431860704700ED00E000E400E03E
:1014D0007047000010B50248FFF7DCFA10BD0000AD
:1014E0002800002010B50168C968026C1180016CE9
:1014F000891C016401464031CA88521ECA80C988CD
:10150000002909D101684A6840239A434A60C18F83
:10151000002901D100F06EF810BD10B50146403130
:10152000CC880368026C012C11D9DB681380026C33
:10153000921C0264CA88921ECA80CA88012A0DD1F0
:1015400002685368012424032343536006E01C7B94
:10155000531C03641470CA88521ECA80C9880029AB
:1015600009D101684A6860239A434A60C18F002903
:1015700001D100F03FF810BD10B5816B02680988F9
:10158000D160816B891C8163C18F491EC187C18F66
:1015900000290AD101684A6880239A434A6046219B
:1015A000095A002901D100F025F810BD10B5C38FEC
:1015B0000268816B022B07D30988D160816B891C7B
:1015C0008163C18F891E05E04B1C83630978117309
:1015D000C18F491EC187C18F00290AD101684A689D
:1015E00080239A434A604621095A002901D100F01C
:1015F00001F810BD70B50446FEF7BEFE0246206835
:1016000041682025A94341606421204600F024F868
:10161000002802D0206E28432066226E2046012139
:101620004030002A04D041772046FFF731FA70BDE0
:10163000427F4177042A204602D0FFF787FB70BD26
:10164000FFF718FB70BD10B5406A00214622115209
:10165000C187FFF71DFA10BDF8B50F460B461546BA
:101660000092032104460022C90200F01BF8202644
:10167000002812D13B46002280212046009500F030
:101680005CF8002809D103213B460022490220468C
:10169000009500F007F8002803D0206E3043206644
:1016A0000320F8BDF8B51D4617460E4604463DE03A
:1016B000032149028E4205D1002F03D1017B6846E8
:1016C00001700078681C31D0002D05D0FEF754FE63
:1016D0000699401AA84229D320684168E022914324
:1016E00041606068C11FFD390CD10121A068C903A8
:1016F000884202D04911884204D120680168402202
:10170000914301600120A16A4003814207D1216811
:101710000A6882430A6021680A6802430A6001205D
:1017200040346077002020770320F8BD206881686E
:101730003140B942BCD10020F8BDF8B51D4617466E
:101740000E46044633E0681C31D0002D05D0FEF76C
:1017500013FE0699401AA84229D320684168E02266
:10176000914341606068C11FFD390CD10121A0681F
:10177000C903884202D04911884204D12068016817
:101780004022914301600120A16A4003814207D1B8
:1017900021680A6882430A6021680A6802430A6075
:1017A000012040346077002020770320F8BD2068B6
:1017B00081683046884304D00020B842C3D100205D
:1017C000F8BD0120F9E7704710B5FEF717FEFFF7E7
:1017D00013FB10BD10B592B0202000900120002412
:1017E000089009946846FEF767FF002800D0FEE7DE
:1017F00007200D9003200E900F94012110940DA846
:10180000FEF756FE002800D0FEE7FEF7FBFE7D2126
:10181000C900FEF78BFCFFF7D7FA0420FFF7C6FAE2
:1018200000221146501EFEF73FFE12B010BD000010
:10183000134801680122114301604168114A1140B7
:1018400041600168104A1140016001680122920460
:101850009143016041683F22120491434160C16A93
:1018600009090901C162016BFF22D432914301636E
:10187000416B4908490041630021816070470000C5
:10188000001002400CB8FF08FFFFF6FE10B502483A
:10189000FFF7C1FB10BD0000CC00002010B50248CE
:1018A000FFF7B9FB10BD00000C010020F0B5026885
:1018B0001A4B0124A4071A4D984203D0A04201D02C
:1018C000A84203D17026B2434E683243154E164FDC
:1018D00098420AD0A04208D0A84206D0134CA04299
:1018E00003D0B04201D0B84204D103242402A24361
:1018F000CC6822438024A2434C69224302608A6858
:10190000C2620A688262984203D0B04201D0B842F3
:1019100001D10969016301214161F0BD002C014041
:101920000004004000440140004801400020004005
:1019300030B58468FF252D021B021343AC430B43D3
:101940002343836030BD826870239A430A43072192
:101950000A438260704730B5036A046A6408640011
:1019600004628469F025AC43120122430A24A34394
:101970000B438261036230BD30B5036A1024A34378
:1019800003628469036A0F252D031203AC432243CB
:10199000A024A343090119438261016230BD10B53F
:1019A000818CC90707D001684A6801235B049A4308
:1019B000836A1A434A60818C890707D501684A689F
:1019C00001231B049A43C36A1A434A60818C490766
:1019D00007D501684A6801239B049A43036B1A43A5
:1019E0004A60818C090707D501684A680123DB0337
:1019F0009A43436B1A434A60818CC90607D5026833
:101A0000916801231B039943836B19439160818C77
:101A1000890607D501688A6801235B039A43C36B73
:101A20001A438A60818C490612D503685A680121DD
:101A30000905046C8A4322435A60026C8A4207D12A
:101A40000268516803235B059943436C1943516055
:101A5000818C090607D501684A680123DB04806C84
:101A60009A4302434A6010BDF8B500260446C66694
:101A7000FEF782FC05461449206888421DD10068A3
:101A8000124F000709D501212B46002249052046A7
:101A9000009700F0B5F800280DD1206800684007D5
:101AA0000BD501212B46002289052046009700F026
:101AB000A7F8002801D00320F8BD20206034607210
:101AC000A07226720020F8BD00380140FFFFFF0120
:101AD000F8B504462369A268E5691A4363691020D2
:101AE0002B43002125681A432B680E463E4F3B408E
:101AF00013432B6023685A6803252D03AA43E56826
:101B00002A435A60236AA26925681A43AB680B27E7
:101B10003F02BB431343AB60344A2568954210D162
:101B2000334A126B9207920F0ED0012A05D0022A77
:101B300005D0032A09D1022007E0042005E008208F
:101B400003E02C4A954200D100200122E369D20330
:101B5000934224D100280CD002280DD0042813D0A1
:101B6000082817D001260A0912010807400F104360
:101B70002FE0FEF74DFD09E061681F4A4808801814
:101B8000FEF7D4FA81B2EEE7FEF752FD616840003D
:101B90004A08F4E76168012248081204EFE70028C8
:101BA00008D0022809D004280BD0082814D0012618
:101BB0003046F8BDFEF72CFD05E061680F4A480885
:101BC0000CE0FEF735FD61684A088018FEF7AEFAB2
:101BD00080B22168C860EBE7616848088018FEF7AA
:101BE000A5FA80B2E860E3E7F369FFEF003801404F
:101BF00000100240004400400024F40000127A006B
:101C0000FFB581B017460E4604460A9D1DE0681CCC
:101C10001BD0002D05D0FEF7AFFB0499401AA84257
:101C200013D920680168FF22A13291430160206826
:101C30008168490849008160202060346072A07288
:101C400000202072032005B0F0BD2068C169304635
:101C5000884304D00020B842D9D00020F3E7012007
:101C6000F9E700000FB410B503A9044B044A029829
:101C700000F018F810BC08BC04B01847DD1E0008BE
:101C80001C00002002E008C8121F08C1002AFAD177
:101C900070477047002001E001C1121F002AFBD1EC
:101CA00070470000FFB58DB00F460546002606E0E0
:101CB00025280AD0109A0F9990476D1C761C287819
:101CC0000028F5D1304611B0F0BD00240121674A4B
:101CD000009400E004436D1C2B780846203B98409C
:101CE0001042F7D128782E2815D1042004436878B3
:101CF0006D1C2A280AD101CF6D1C00900BE00099C1
:101D00000A225143303940186D1C00902878014652
:101D100030390929F3D92878692843D006DC00280E
:101D2000D0D063280BD0642804D13BE073280FD0B7
:101D300075284CD0109A0F999047761C94E038780B
:101D4000694608720020487202A80190012003E051
:101D5000386801900020C0433F1D61070CD5002466
:101D600000E0641C00998C420FDA8442F9DB01998F
:101D7000095D0029F5D108E0002400E0641C8442DC
:101D8000FCDB0199095D0029F8D1361907E00198BB
:101D900001990078491C0191109A0F999047641E8F
:101DA000F5D261E00A20019001CF002802DA40421A
:101DB0002D2102E0210504D52B216A461172012153
:101DC00003E0E10701D02021F7E70C9104E00A20AD
:101DD000019001CF00210C910BA90B9108E0019912
:101DE000FEF7A4F90A460B993032491E0B910A708E
:101DF0000028F4D10B9803A9081A2030019060073D
:101E000001D5009801E0012000900199884203DD8E
:101E100001460198081A00E000200024009006E026
:101E200002A8109A005D0F999047641C761C0C98CC
:101E30008442F5DB04E0109A30200F999047761C1D
:101E40000099481E00900029F5DC08E00B980B99DA
:101E50000078491C0B91109A0F999047761C0199B4
:101E6000481E01900029F1DC6D1C28E709280100BB
:101E700010B5064A064C91784B00E052491CC8B296
:101E80009070082801D30020907010BD040000203D
:101E9000240200200902014308B27047002800DA3A
:101EA0004042002801DC07487047402802DBFF2041
:101EB000F5307047BD21C94348430349401880B2FB
:101EC00070470000FFFF00009231000010B502498A
:101ED0000860FFF711F810BD0000002013B50A23B9
:101EE000012269460248FFF7B3F900981CBD0000C3
:101EF0004C01002000200C4A01464B00D35E491CD7
:101F000018180829F9DB411E072901D2082006E02C
:101F1000002804DA4142082901DA0720C043C1172A
:101F2000490F0818C01070472402002070B54406FD
:101F3000C109640EC901102C1AD20E4D285D00286B
:101F400016D0002910D0022812D1032C02D0062C62
:101F500008D104E00748183800F046F802E00648C7
:101F600000F06CF9012002E0012801D1022028557F
:101F700070BD0000140200200C00002070B5154652
:101F80000E46044600F022F8002801D0012070BD62
:101F90002178606846542178A06845542078A1785B
:101FA000401CFEF7C3F82170002070BD70B50D46CF
:101FB00004468170284600F0C1F86060284600F0B1
:101FC000BDF8A060204600F00FF870BD10B50446C3
:101FD00081780078401CFEF7A9F86078814201D131
:101FE000012010BD002010BD10B504460020207057
:101FF0006070A1786068FEF7C8F8A178A068FEF765
:10200000C4F810BD1CB5FEF701FAFFF7E3FBFFF7BC
:1020100085F9FFF7D5F9FFF71BFAFFF7EFF9384815
:10202000364900242F25846022C08460C46035496D
:10203000046141600838FEF709FF002800D0FEE780
:102040002F4831494038846022C084602F49C460E1
:102050004160802101610838FEF7F8FE002800D0B9
:10206000FEE7012000902A4D019000232A7829499B
:1020700029A0FFF7F7FD22488038FFF727FF00F07F
:1020800055F91F481021F030FFF790FF2846102126
:10209000083000F0A2F81A482021B030FEF775F899
:1020A000174A17482023D032D11AE438FEF7E4FD4E
:1020B00002201E4900900B4601221D4800F056F9EF
:1020C0000F48FEF725FF0E484038FEF721FF3F245A
:1020D000E4432046FFF7E2FE0246214615A0FFF743
:1020E000C1FD641C402CF4DB6878002801D000F0AE
:1020F00065F93220FEF78AF8F6E700000048014053
:102100000C0100201027000000440140FFFF0000E8
:10211000040000203C24000825730A7265762564BB
:10212000207625642E25642E25640A0000140048BC
:102130003402002025642025640A0000F0B50B302D
:10214000C108C900144F0026144A0FE003688B42EF
:102150000BD38B4205D95C1A4318456830C3083B42
:1021600000E04368136002C004E0021D106800280C
:10217000ECD13046002803D13868002801D0002077
:10218000F0BD064A06481060064A121AD208D2006C
:1021900044C001203860D7E7240000202000002040
:1021A0004C0200204804002070B50D46044600F0A3
:1021B00020F8002801D0012070BD20780C22616831
:1021C000504308182946FDF7C7FF2078A178401C26
:1021D000FDF7ACFF2170002070BD10B50446817082
:1021E0000C204843FFF7AAFF6060204600F026F865
:1021F00010BD10B5044681780078401CFDF796FFAD
:102200006078814201D1012010BD002010BD4178CD
:102210000278914201D10020704740680C2251435E
:102220004018704710B5044640782178884204D0A1
:10223000A178401CFDF77AFF617010BD10B5002138
:102240000170417081780C2251434068FDF79DFF79
:1022500010BD000070B50446807809280FD008280A
:102260002AD001282FD0022808D10325605D00283C
:1022700004D0FFF75BFE6D1C202DF7DB70BD61798C
:102280002079FFF707FE274A1080E179A079FFF750
:1022900001FE5080207A234940429080607B9071FB
:1022A000A07B1072E07BD071207C5072607C9072B9
:1022B0001D48FFF779FF70BD1A48A27921790C38C3
:1022C000FFF75CFE70BD174820214C38FDF75DFF1D
:1022D0001448CD214C38017061784170802585709B
:1022E0000221C170104908220839097801710021C2
:1022F000417101218171C171002104465834635C30
:10230000002B0BD0022B02D0012B02D004E0815411
:1023100002E00B462B438354521CD2B2491C1029B5
:10232000EDDB70BD080200200C00002005480021F4
:10233000C16601674167816701216C30C17081719D
:1023400070470000A801002010B5817B491E890755
:10235000890F817300F01AF810BD10B5817B491CFC
:102360008907890F817300F011F810BD10B5029C28
:10237000016082808360848100F001F810BD10B597
:102380000021817300F002F810BD000070B5044612
:10239000807B09490D5CA1882068EA0700D00122F2
:1023A000FDF7E4FFA807A189A06801D5012200E09C
:1023B0000022FDF7DBFF70BD3824000812A0FFF7F4
:1023C00051FC144D0024295D13A0FFF74BFC641C45
:1023D000202CF8DB11A0FFF745FC0024FF25134E4D
:1023E000013529463046FDF7BDFF6420FDF70EFF9D
:1023F000641C642CF5DBBFF34F8F0E490C48C8609A
:10240000BFF34F8F00BFFDE7535049204552524F55
:10241000520A0000DC010020256420000A72656277
:102420006F6F74696E672E2E2E0A0000000400483C
:102430000400FA0500ED00E00001030255534234A8
:1024400056432050726F746F636F6C20426F6172DD
:10245000640A5175616420656E636F6465722074EF
:102460006573740A64656B754E756B656D203230EB
:1024700032320000000000000000000102030406E8
:10248000070809000000000102030400AC24000852
:102490000000002028000000841C0008D42400084C
:1024A0002800002020080000941C00080000000004
:1024B000000000000000000000000000000000001C
:1024C0000000000000127A00000000000000000080
:0424D0000000000008
:04000005080000C12E
:00000001FF
